:020000040000FA
:080000008A1500278A157729F3
:08000800F000030E8301F1007A
:100010000408F2000A08B0008A151108C8008C18FC
:10002000FC220D1B8A2230088A0072088400710E9F
:080030008300F00E700E0900C0
:041000000034003484
:0C1004007E1A442804303B02031C4C34CC
:1010100022083D3C031D032908308A0020082106D0
:10102000F300E039031D493420088A159A2321086A
:101030009A233A309A2320309A2308308A00730882
:10104000243E03188A0A8200493449344628493428
:101050004B284934493449346428493449344934A3
:101060004934642864286428502849344934493470
:1010700055285A2849344934493449344934493483
:1010800049345F28493449347E1255342008503C95
:1010900003198A2849342008563C031997284934F3
:1010A0002008473C0319F52849342008443C03191B
:1010B0008C2849342008453C0319EB284934200882
:1010C000493C0319DD28493420084C3C031D4934B0
:1010D0007F20031C080023088A159A238A154130B3
:1010E0002102F3000830F3184030B40003107318E5
:1010F000B40D0608231C06093405860608000310F3
:101100003B08043A031D4C342308313C013C0318CE
:1011100008004F348A15D72B3B08053C031D4C347F
:101120004C2103180800840000088A15902B3B0806
:10113000043C031D4C342308393C093C031C4F3448
:10114000033EF300E03883169D008312E0304B0528
:101150007304CB00AD208A15F12BF30000308A1503
:1011600041228A15831203178D0073088316031713
:101170000C14831203170C060319CA288C06831655
:1011800003170C158B1355308D00AA308D008C146D
:101190008B170C1183120313730808000310F4005B
:1011A0000130F4180430F3007418F30D7419F30EC1
:1011B000F40E740D740D1F3908007F20031C080005
:1011C00020302318CB04FF3A231CCB054B08AD205D
:1011D00023088A159A2B7F20031C0800031DC717BC
:1011E0000319C71323088A159A2B3B08043C031DD7
:1011F0004C342308523C031D4F34031386108316CE
:1012000086108A1100283B08083A031D4C34203010
:1012100084004D2103180800F9004D21031808002F
:10122000FA004D2103180800FB004D2103180800A7
:10123000FC000130C600451445160830791B1030FB
:10124000BE002230BD0083168C148312F930910049
:1012500012150530791FC2008A15BD2B233084007A
:1012600008000008393C093C031C4A29F300840AA1
:101270000008393C093C031C4829B2001A307302AB
:1012800003185234730869213207031C362952347B
:101290007308080003144C342E215621031808004B
:1012A000F300F30E5621031C7304080030300002D3
:1012B000031C4A29F63E031C6529DF39F93E031C4D
:1012C0004A29FA3E03184C34063E0A3E840A0310AB
:0E12D0000800B300B307B30DB307330D0800D9
:0212DE006400AA
:1012E000061D6F2998011A088A1500278A1503130D
:1012F000831286010516831660308F00E730850063
:1013000027308600FE01031EFE15D5308100F9301E
:1013100092008312003092003130900081010B1155
:1013200064000B1D9029033083169C0007309B003E
:101330001930990018151812981683129817181654
:1013400041309F00203084005030FD00803080010B
:1013500084068001840AFD0BA72900304D22CB00B2
:10136000E03883169D000D178C14830183161C0E24
:1013700083120D130C39C500450DE7388500FF3089
:1013800086000B178B173D30C00004308A158B2365
:101390008A156400BF08031D30224418052247192E
:1013A0000A220B191D220C1B5B2218196F298C1A9B
:1013B000F221C9293B08203E84001A08C4190800FC
:1013C00080000A3A03190800073A0319EC293B0880
:1013D000013E831CBB000800BB0803190800800104
:1013E000C4150800981CF729181218167E16DA2161
:1013F000C41D08008A150220BB01C4118A150038DB
:10140000031D75238C238A1508008A15B0238A15BD
:101410004410080047116430471C192A5830C71C73
:10142000162A41087A3C031C08005F308A15752390
:1014300067308A158B238A1508000B11C00B252AEB
:101440003D30C000C20B08008511121D1F158A1502
:1014500049090319C901C908031DC9238A150800D0
:101460000C1E08003C08A03E8400000899000408F7
:1014700080008013BC0A50303C060319BC01BF0336
:101480000800831603178C1C0800831203138C1E9C
:10149000412AF400DA217408412A41228C01831286
:1014A00003178D00831603170C14831203170C08FF
:1014B0008312031308000C131E084106C1064106DF
:1014C0004102031C003CFC39031D080041087A3C22
:1014D000031C762A4108733C683C0318C41C0800AE
:1014E000C41034308A158B238A150800C4180800EC
:1014F000C4141C308A158B238A1512110B13831602
:101500001C121C0E83120D130B1745060C39C50651
:04151000C701080007
:0C15140083161C0E83120D1345060C39C3
:1015200003190800C50604390319C71D9A2AFF309C
:10153000C9000800031DC719A22AC715BD08031951
:10154000451AB82ABD080319D32A03304602031CE2
:101550005D2B83161C0D8312C719803EBD0BC12A5B
:10156000031C622BC51B662B4414C7111211D02A11
:10157000BD01451218304718083005061839850690
:10158000C92A80300318C506F80DF70DF60DF50DC4
:101590004513C601480891020630031C91028C10C5
:1015A0006430810008001219E02AC908031DD02AFE
:1015B0002A3091001215C60183168C148312D02A8A
:1015C0000A3046020318C92A83161C0D8312C71954
:1015D000803E031CD02A83161C1E0310831203189E
:1015E000C718F42AC7144715C6080319B62A2130AC
:1015F000BD00C5134513C92A8C10C60A451A062B0F
:10160000BD080319282BC619642B080046180800CA
:10161000BD080319202B0301451C18304718103A48
:1016200005063E058506C618252B45100314FC0D3E
:10163000FB0DFA0DF90D03184514C601BD03080092
:10164000121145123E1AC51608000130C5060800E1
:10165000C71D08004608143C03193D2B50304602B4
:10166000031C08001211C71183161C1E03108312DD
:10167000031C0800C71447150800451DC71F0800B4
:10168000831610309C061C1E03101C0E83120D13B3
:1016900045060C39C5060318542B4715C71C08000E
:1016A0004710C710051608004718592B4714051294
:1016B0000800C71408004517D02A451BCB1A5B2B1E
:1016C0000130672B0230672B0330672B0430C908C9
:1016D0000319C9001211BD01C601451249090319B8
:0A16E000732B7A30CA008A15D02A55
:0616EA008A1541228A1559
:1016F000831203178D00802B9A23831203178D0A00
:10170000831603170C14831203170C088312031398
:10171000031D7C2B080075230D309A230A309A2B69
:10172000F400740E942374080F39F63E0318073E34
:101730000A3E303EBF0803190C1EA02B990000344E
:1017400084003C083F07B03E031C503EA03E040608
:101750008406040680003F08503A031DBF0A003487
:101760005430751B42309A237508902376089023D5
:1017700077089023780890238C2B5230791B4130C6
:101780009A23790890237A0890237B0890237C0879
:10179000902B471908006E307523490890238C233D
:1017A0004530491CB323C9010800070D992B3B089C
:1017B000043A031D4C342308413A03190234153A04
:1017C0000319EA2B023A0319F02B4F3423089A230A
:1017D0003D309A2BE6234B0EF300F30CF30CD52B84
:0817E000E6234B08FD3E942BAB
:101E0000031E08008B138316031360308F002730E6
:101E10008600E730850007309B00E6309D000630E5
:101E20009C00D73081001930990026309800831229
:101E300098171816FF30860081010130E327C2276A
:101E40001030E3278C1E0800C827031D08008317E5
:101E500010308400F001C8270319282F0B3A03190A
:101E6000392F013A0319C82772088000F007840A45
:101E70002B2FF008031D822F031712088D00130863
:101E80008F00143084001108F1000F308A00100810
:101E9000083C083C031C822F8207592F5F2F872F95
:101EA000992FA12FAC2F822F822FED2F0101000F30
:101EB000FF0F56308D000F308F00123084008316D4
:101EC0008C170C140000000083120C088000840A98
:101ED0000E088000840A8D0A03198F0AF10B5F2F08
:101EE00010300402F1000F30C227F00110308400DE
:101EF0000008F007840AB527F10B782F7009013E1E
:101F0000B527C2270313C8270319282F822F84302F
:101F1000D127FC308D050430F40000088C00840AC1
:101F200000088E00840AD527F40B8D2FF10B872F24
:101F3000722F9430D1271F308D04D527F10B992FA4
:101F4000722F83168C010C1483120C088000840AF3
:101F50008D0AF10BA12F702F0430D12700088C00BF
:101F6000840AD527F10BAC2F722FF3000F3A031917
:101F7000BF2F0B3A0319BF2F013A031DC12F0530A4
:101F8000C2277308640003130C1EC42F9900043485
:101F90009818ED2F64008C1ECA2F1A08F2000F3A11
:101FA000080083168C0083120800640083165530E5
:101FB0008D00AA308D008C148C18DC2F83128D0AB2
:101FC00003198F0A013464008C1A08000B1DE32FDB
:101FD0000B11FF3E031DE32F0434031386108316F9
:101FE0008610FF308500860081009B0007309C0032
:101FF00098019901830198018B018A0164000028EE
:02400E00742F0D
:02401000FF3F70
:104200002600000041003D004F00700065006E0078
:1042100054006800650072006D00200049006E00C7
:104220007400650072006600610063006500200094
:1042300031002E003100000054006800650072005B
:104240006D006F0073007400610074002000640052
:104250006900730063006F006E006E00650063000C
:10426000740065006400000054006800650072007E
:104270006D006F0073007400610074002000630023
:104280006F006E006E0065006300740065006400DE
:1042900000004E00470000005300450000004200AF
:1042A000560000004F00520000004F004500000083
:1042B0004D0065006400690075006D000000480055
:1042C00069006700680000004C006F007700200064
:1042D00070006F00770065007200000045007200FA
:1042E00072006F00720020000000310037003A00B9
:1042F000350039002000320030002D003100300040
:104300002D00320030003100350000003400200064
:084310004D0048007A00000096
:00000001FF
